Microchip MPLAB XC8 Compiler V2.41

Linker command line:

-W-3 \
  --edf=E:/Program Files/Microchip/MPLABX/v6.15/packs/Microchip/PIC18F-Q_DFP/1.20.405/xc8\pic\dat\20230718171817_en.msgs \
  -pivt0x8=08h -cn -h+dist/default/production\I2CPwm2.X.production.sym \
  --cmf=dist/default/production\I2CPwm2.X.production.cmf -z -Q18F06Q40 \
  -oC:\Users\stephen\AppData\Local\Temp\xcAs34s.\driver_tmp_3.o \
  --defsym=__MPLAB_BUILD=1 --fixupoverflow=error \
  -Mdist/default/production/I2CPwm2.X.production.map \
  --md=C:\Users\stephen\AppData\Local\Temp\xcAs34s.\driver_tmp_0.dat -E1 \
  -ver=XC8 Compiler --acfsm=1493 -ACODE=00h-0FFFFh -ACONST=00h-0FFFFh \
  -ASMALLCONST=01600h-016FFhx234 -AMEDIUMCONST=01600h-0FFFFh \
  -ACOMRAM=0501h-055Fh -AABS1=0500h-014FFh -ABIGRAM=0501h-014FFh \
  -ARAM=0560h-05FFh,0600h-06FFhx15 -ABANK5=0560h-05FFh -ABANK6=0600h-06FFh \
  -ABANK7=0700h-07FFh -ABANK8=0800h-08FFh -ABANK9=0900h-09FFh \
  -ABANK10=0A00h-0AFFh -ABANK11=0B00h-0BFFh -ABANK12=0C00h-0CFFh \
  -ABANK13=0D00h-0DFFh -ABANK14=0E00h-0EFFh -ABANK15=0F00h-0FFFh \
  -ABANK16=01000h-010FFh -ABANK17=01100h-011FFh -ABANK18=01200h-012FFh \
  -ABANK19=01300h-013FFh -ABANK20=01400h-014FFh \
  -ASFR=00h-0FFhx4,0400h-045Fh,0460h-04FFh,01500h-015FFh \
  -ABIGSFR=00h-04FFh,01500h-015FFh -ACONFIG=0300000h-0300011h \
  -AIDLOC=0200000h-020003Fh -AEEDATA=0380000h-03801FFh -peeprom_data=EEDATA \
  -preset_vec=00h -ppowerup=CODE,init -pramtop=01600h \
  -psmallconst=SMALLCONST -pmediumconst=MEDIUMCONST -pconst=CONST \
  -AFARRAM=00h-00h \
  -prdata=COMRAM,nvrram=COMRAM,nvbit=COMRAM,rbss=COMRAM,rbit=COMRAM \
  -pfarbss=FARRAM,fardata=FARRAM,nvFARRAM=FARRAM \
  -pintsave_regs=BIGRAM,bigbss=BIGRAM,bigdata=BIGRAM -pbss=RAM \
  -pidata=CODE,irdata=CODE,ibigdata=CODE,ifardata=CODE -prparam=COMRAM \
  C:\Users\stephen\AppData\Local\Temp\xcAs34s.\driver_tmp_9.o \
  dist/default/production\I2CPwm2.X.production.o 

Object code version is 3.11

Machine type is 18F06Q40



                Name                               Link     Load   Length Selector   Space Scale
C:\Users\stephen\AppData\Local\Temp\xcAs34s.\driver_tmp_9.o
                config                           300000   300000        9        0       4
                init                                 1A       1A        4        4       0
                reset_vec                             0        0        4        0       0
dist/default/production\I2CPwm2.X.production.o
                config                           300000   300000        9        0       4
                ivt0x8                                8        8       12        4       0
                text54                              7B6      7B6        8        4       0
                text53                              7AE      7AE        8        4       0
                text52                              57A      57A       2E        4       0
                text51                              7D6      7D6        6        4       0
                text50                              7A6      7A6        8        4       0
                text49                              69A      69A       16        4       0
                text48                              684      684       16        4       0
                text47                              66E      66E       16        4       0
                text46                              658      658       16        4       0
                text45                              642      642       16        4       0
                text44                              7D0      7D0        6        4       0
                text43                              4CE      4CE       50        4       0
                text42                              54C      54C       2E        4       0
                text41                              7CA      7CA        6        4       0
                text40                              6FA      6FA        E        4       0
                text39                              79E      79E        8        4       0
                text38                              3B4      3B4       64        4       0
                text37                              51E      51E       2E        4       0
                text36                               1E       1E      132        4       0
                text35                              150      150       AC        4       0
                text34                              6E8      6E8       12        4       0
                text33                              6B0      6B0       14        4       0
                text32                              794      794        A        4       0
                text31                              78A      78A        A        4       0
                text30                              780      780        A        4       0
                text29                              776      776        A        4       0
                text28                              6D6      6D6       12        4       0
                text27                              6C4      6C4       12        4       0
                text26                              76C      76C        A        4       0
                text25                              762      762        A        4       0
                text24                              418      418       5E        4       0
                text23                              7C4      7C4        6        4       0
                text22                              7BE      7BE        6        4       0
                text21                              7E8      7E8        4        4       0
                text20                              7E4      7E4        4        4       0
                text19                              7E0      7E0        4        4       0
                text18                              626      626       1C        4       0
                text17                              7DC      7DC        4        4       0
                text16                              60A      60A       1C        4       0
                text15                              346      346       6E        4       0
                text14                              5EE      5EE       1C        4       0
                text13                              758      758        A        4       0
                text12                              74E      74E        A        4       0
                text11                              744      744        A        4       0
                text10                              2D8      2D8       6E        4       0
                text9                               73A      73A        A        4       0
                text8                               730      730        A        4       0
                text7                               726      726        A        4       0
                text6                               26A      26A       6E        4       0
                text5                               71C      71C        A        4       0
                text4                               712      712        A        4       0
                text3                               708      708        A        4       0
                text2                               1FC      1FC       6E        4       0
                text1                               5CC      5CC       22        4       0
                text0                               476      476       58        4       0
                cstackCOMRAM                        527      527        A      501       1
                bssCOMRAM                           501      501       14      501       1
                cinit                               5A8      5A8       24        4       0
                nvCOMRAM                            515      515       12      501       1

TOTAL           Name                               Link     Load   Length     Space
        CLASS   CODE           
                init                                 1A       1A        4         0
                reset_vec                             0        0        4         0
                ivt0x8                                8        8       12         0
                text54                              7B6      7B6        8         0
                text53                              7AE      7AE        8         0
                text52                              57A      57A       2E         0
                text51                              7D6      7D6        6         0
                text50                              7A6      7A6        8         0
                text49                              69A      69A       16         0
                text48                              684      684       16         0
                text47                              66E      66E       16         0
                text46                              658      658       16         0
                text45                              642      642       16         0
                text44                              7D0      7D0        6         0
                text43                              4CE      4CE       50         0
                text42                              54C      54C       2E         0
                text41                              7CA      7CA        6         0
                text40                              6FA      6FA        E         0
                text39                              79E      79E        8         0
                text38                              3B4      3B4       64         0
                text37                              51E      51E       2E         0
                text36                               1E       1E      132         0
                text35                              150      150       AC         0
                text34                              6E8      6E8       12         0
                text33                              6B0      6B0       14         0
                text32                              794      794        A         0
                text31                              78A      78A        A         0
                text30                              780      780        A         0
                text29                              776      776        A         0
                text28                              6D6      6D6       12         0
                text27                              6C4      6C4       12         0
                text26                              76C      76C        A         0
                text25                              762      762        A         0
                text24                              418      418       5E         0
                text23                              7C4      7C4        6         0
                text22                              7BE      7BE        6         0
                text21                              7E8      7E8        4         0
                text20                              7E4      7E4        4         0
                text19                              7E0      7E0        4         0
                text18                              626      626       1C         0
                text17                              7DC      7DC        4         0
                text16                              60A      60A       1C         0
                text15                              346      346       6E         0
                text14                              5EE      5EE       1C         0
                text13                              758      758        A         0
                text12                              74E      74E        A         0
                text11                              744      744        A         0
                text10                              2D8      2D8       6E         0
                text9                               73A      73A        A         0
                text8                               730      730        A         0
                text7                               726      726        A         0
                text6                               26A      26A       6E         0
                text5                               71C      71C        A         0
                text4                               712      712        A         0
                text3                               708      708        A         0
                text2                               1FC      1FC       6E         0
                text1                               5CC      5CC       22         0
                text0                               476      476       58         0
                cinit                               5A8      5A8       24         0

        CLASS   CONST          

        CLASS   SMALLCONST     

        CLASS   MEDIUMCONST    

        CLASS   COMRAM         
                cstackCOMRAM                        527      527        A         1
                bssCOMRAM                           501      501       14         1
                nvCOMRAM                            515      515       12         1

        CLASS   ABS1           

        CLASS   BIGRAM         

        CLASS   RAM            

        CLASS   BANK5          

        CLASS   BANK6          

        CLASS   BANK7          

        CLASS   BANK8          

        CLASS   BANK9          

        CLASS   BANK10         

        CLASS   BANK11         

        CLASS   BANK12         

        CLASS   BANK13         

        CLASS   BANK14         

        CLASS   BANK15         

        CLASS   BANK16         

        CLASS   BANK17         

        CLASS   BANK18         

        CLASS   BANK19         

        CLASS   BANK20         

        CLASS   SFR            

        CLASS   BIGSFR         

        CLASS   CONFIG         
                config                           300000   300000        9         4

        CLASS   IDLOC          

        CLASS   EEDATA         

        CLASS   FARRAM         

        CLASS   HEAP           

        CLASS   STACK          



SEGMENTS        Name                           Load    Length   Top    Selector   Space  Class

                reset_vec                      000000  000004  000004         0       0  CODE    
                ivt0x8                         000008  0007E4  0007EC         4       0  CODE    
                bssCOMRAM                      000501  000030  000531       501       1  COMRAM  


UNUSED ADDRESS RANGES

        Name                Unused          Largest block    Delta
        BANK10           000A00-000AFF              100
        BANK11           000B00-000BFF              100
        BANK12           000C00-000CFF              100
        BANK13           000D00-000DFF              100
        BANK14           000E00-000EFF              100
        BANK15           000F00-000FFF              100
        BANK16           001000-0010FF              100
        BANK17           001100-0011FF              100
        BANK18           001200-0012FF              100
        BANK19           001300-0013FF              100
        BANK20           001400-0014FF              100
        BANK5            000560-0005FF               A0
        BANK6            000600-0006FF              100
        BANK7            000700-0007FF              100
        BANK8            000800-0008FF              100
        BANK9            000900-0009FF              100
        BIGRAM           000531-0014FF              FCF
        BIGSFR           000000-0004FF              500
                         001500-0015FF              100
        CODE             000004-000007                4
                         0007EC-00FFFF             F814
        COMRAM           000531-00055F               2F
        CONFIG           300009-300011                9
        CONST            000004-000007                4
                         0007EC-00FFFF             F814
        EEDATA           380000-3801FF              200
        IDLOC            200000-20003F               40
        MEDIUMCONST      001600-00FFFF             EA00
        RAM              000560-0014FF              100
        SFR              000000-0004FF              100
                         001500-0015FF              100
        SMALLCONST       001600-00FFFF              100

                                  Symbol Table

I2C1_SlaveDefRdInterruptHandler@i                             cstackCOMRAM 000527
I2C1_SlaveDefWrInterruptHandler@i                             cstackCOMRAM 000528
I2C1_SlaveSendTxData@data                                     cstackCOMRAM 000527
I2C1_SlaveSetAddrIntHandler@handler                           cstackCOMRAM 00052D
I2C1_SlaveSetBusColIntHandler@handler                         cstackCOMRAM 00052D
I2C1_SlaveSetCounter@counter                                  cstackCOMRAM 000527
I2C1_SlaveSetIsrHandler@handler                               cstackCOMRAM 00052D
I2C1_SlaveSetReadIntHandler@handler                           cstackCOMRAM 00052D
I2C1_SlaveSetSlaveAddr@slaveAddr                              cstackCOMRAM 00052D
I2C1_SlaveSetSlaveMask@maskAddr                               cstackCOMRAM 00052D
I2C1_SlaveSetWrColIntHandler@handler                          cstackCOMRAM 00052D
I2C1_SlaveSetWriteIntHandler@handler                          cstackCOMRAM 00052D
IVTBASEH                                                      (abs)        00045E
IVTBASEL                                                      (abs)        00045D
IVTBASEU                                                      (abs)        00045F
PWM1_16BIT_Period_SetInterruptHandler@InterruptHandler        cstackCOMRAM 00052D
PWM1_16BIT_Slice1Output1_SetInterruptHandler@InterruptHandler cstackCOMRAM 00052D
PWM1_16BIT_Slice1Output2_SetInterruptHandler@InterruptHandler cstackCOMRAM 00052D
PWM2_16BIT_Period_SetInterruptHandler@InterruptHandler        cstackCOMRAM 00052D
PWM2_16BIT_Slice1Output1_SetInterruptHandler@InterruptHandler cstackCOMRAM 00052D
PWM2_16BIT_Slice1Output2_SetInterruptHandler@InterruptHandler cstackCOMRAM 00052D
PWM3_16BIT_Period_SetInterruptHandler@InterruptHandler        cstackCOMRAM 00052D
PWM3_16BIT_Slice1Output1_SetInterruptHandler@InterruptHandler cstackCOMRAM 00052D
PWM3_16BIT_Slice1Output2_SetInterruptHandler@InterruptHandler cstackCOMRAM 00052D
_ACTCON                                                       (abs)        0000AC
_ANSELA                                                       (abs)        000400
_ANSELC                                                       (abs)        000410
_I2C1ADB0                                                     (abs)        00028E
_I2C1ADR0                                                     (abs)        000290
_I2C1ADR1                                                     (abs)        000291
_I2C1ADR2                                                     (abs)        000292
_I2C1ADR3                                                     (abs)        000293
_I2C1BAUD                                                     (abs)        00029D
_I2C1CNTH                                                     (abs)        00028D
_I2C1CNTL                                                     (abs)        00028C
_I2C1CON0                                                     (abs)        000294
_I2C1CON0bits                                                 (abs)        000294
_I2C1CON1                                                     (abs)        000295
_I2C1CON1bits                                                 (abs)        000295
_I2C1CON2                                                     (abs)        000296
_I2C1ERRbits                                                  (abs)        000297
_I2C1PIEbits                                                  (abs)        00029B
_I2C1PIR                                                      (abs)        00029A
_I2C1PIRbits                                                  (abs)        00029A
_I2C1RXB                                                      (abs)        00028A
_I2C1SCLPPS                                                   (abs)        000271
_I2C1SDAPPS                                                   (abs)        000270
_I2C1STAT0bits                                                (abs)        000298
_I2C1STAT1bits                                                (abs)        000299
_I2C1TXB                                                      (abs)        00028B
_I2C1_Initialize                                              text18       000626
_I2C1_InterruptHandler                                        bssCOMRAM    00050F
_I2C1_Isr                                                     text36       00001E
_I2C1_Open                                                    text24       000418
_I2C1_SlaveAddrCallBack                                       text52       00057A
_I2C1_SlaveAddrInterruptHandler                               bssCOMRAM    000509
_I2C1_SlaveBusColInterruptHandler                             bssCOMRAM    000507
_I2C1_SlaveClearBuff                                          text51       0007D6
_I2C1_SlaveClearIrq                                           text50       0007A6
_I2C1_SlaveDefAddrInterruptHandler                            text53       0007AE
_I2C1_SlaveDefBusColInterruptHandler                          (abs)        000000
_I2C1_SlaveDefRdInterruptHandler                              text43       0004CE
_I2C1_SlaveDefWrColInterruptHandler                           (abs)        000000
_I2C1_SlaveDefWrInterruptHandler                              text38       0003B4
_I2C1_SlaveEnableIrq                                          text34       0006E8
_I2C1_SlaveGetAddr                                            text54       0007B6
_I2C1_SlaveGetRxData                                          text44       0007D0
_I2C1_SlaveIsAddr                                             text49       00069A
_I2C1_SlaveIsRead                                             text48       000684
_I2C1_SlaveIsRxBufFull                                        text47       00066E
_I2C1_SlaveIsStop                                             text46       000658
_I2C1_SlaveIsTxBufEmpty                                       text45       000642
_I2C1_SlaveOpen                                               text33       0006B0
_I2C1_SlaveRdCallBack                                         text42       00054C
_I2C1_SlaveRdInterruptHandler                                 bssCOMRAM    00050D
_I2C1_SlaveReleaseClock                                       text41       0007CA
_I2C1_SlaveSendTxData                                         text39       00079E
_I2C1_SlaveSetAddrIntHandler                                  text32       000794
_I2C1_SlaveSetBusColIntHandler                                text31       00078A
_I2C1_SlaveSetCounter                                         text40       0006FA
_I2C1_SlaveSetIsrHandler                                      text30       000780
_I2C1_SlaveSetReadIntHandler                                  text29       000776
_I2C1_SlaveSetSlaveAddr                                       text28       0006D6
_I2C1_SlaveSetSlaveMask                                       text27       0006C4
_I2C1_SlaveSetWrColIntHandler                                 text26       00076C
_I2C1_SlaveSetWriteIntHandler                                 text25       000762
_I2C1_SlaveWrCallBack                                         text37       00051E
_I2C1_SlaveWrColInterruptHandler                              bssCOMRAM    000505
_I2C1_SlaveWrInterruptHandler                                 bssCOMRAM    00050B
_I2C1_ZeroBuff                                                text23       0007C4
_I2C1_ZeroBuffer                                              text22       0007BE
_INLVLA                                                       (abs)        000404
_INLVLC                                                       (abs)        000414
_INTCON0bits                                                  (abs)        0004D6
_INTERRUPT_Initialize                                         text17       0007DC
_INTERRUPT_InterruptManager                                   text35       000150
_LATA                                                         (abs)        0004BE
_LATC                                                         (abs)        0004C0
_ODCONA                                                       (abs)        000402
_ODCONC                                                       (abs)        000412
_OSCCON1                                                      (abs)        0000AD
_OSCCON3                                                      (abs)        0000AF
_OSCEN                                                        (abs)        0000B3
_OSCFRQ                                                       (abs)        0000B1
_OSCILLATOR_Initialize                                        text16       00060A
_OSCTUNE                                                      (abs)        0000B0
_PIE4bits                                                     (abs)        0004AC
_PIE5bits                                                     (abs)        0004AD
_PIE7bits                                                     (abs)        0004AF
_PIN_MANAGER_Initialize                                       text15       000346
_PIR4bits                                                     (abs)        0004B7
_PIR5bits                                                     (abs)        0004B8
_PIR7bits                                                     (abs)        0004BA
_PMD0                                                         (abs)        000063
_PMD1                                                         (abs)        000064
_PMD2                                                         (abs)        000065
_PMD3                                                         (abs)        000066
_PMD4                                                         (abs)        000067
_PMD5                                                         (abs)        000068
_PMD_Initialize                                               text14       0005EE
_PWM1CLK                                                      (abs)        000461
_PWM1CON                                                      (abs)        000469
_PWM1CONbits                                                  (abs)        000469
_PWM1CPRE                                                     (abs)        000465
_PWM1ERS                                                      (abs)        000460
_PWM1GIE                                                      (abs)        000468
_PWM1GIEbits                                                  (abs)        000468
_PWM1GIR                                                      (abs)        000467
_PWM1GIRbits                                                  (abs)        000467
_PWM1LDS                                                      (abs)        000462
_PWM1PIPOS                                                    (abs)        000466
_PWM1PRH                                                      (abs)        000464
_PWM1PRL                                                      (abs)        000463
_PWM1S1CFG                                                    (abs)        00046A
_PWM1S1P1H                                                    (abs)        00046C
_PWM1S1P1L                                                    (abs)        00046B
_PWM1S1P2H                                                    (abs)        00046E
_PWM1S1P2L                                                    (abs)        00046D
_PWM1_16BIT_Enable                                            text21       0007E8
_PWM1_16BIT_Initialize                                        text10       0002D8
_PWM1_16BIT_Period_DefaultInterruptHandler                    (abs)        000000
_PWM1_16BIT_Period_InterruptHandler                           nvCOMRAM     000515
_PWM1_16BIT_Period_SetInterruptHandler                        text13       000758
_PWM1_16BIT_Slice1Output1_DefaultInterruptHandler             (abs)        000000
_PWM1_16BIT_Slice1Output1_InterruptHandler                    nvCOMRAM     000519
_PWM1_16BIT_Slice1Output1_SetInterruptHandler                 text12       00074E
_PWM1_16BIT_Slice1Output2_DefaultInterruptHandler             (abs)        000000
_PWM1_16BIT_Slice1Output2_InterruptHandler                    nvCOMRAM     000517
_PWM1_16BIT_Slice1Output2_SetInterruptHandler                 text11       000744
_PWM2CLK                                                      (abs)        000470
_PWM2CON                                                      (abs)        000478
_PWM2CONbits                                                  (abs)        000478
_PWM2CPRE                                                     (abs)        000474
_PWM2ERS                                                      (abs)        00046F
_PWM2GIE                                                      (abs)        000477
_PWM2GIEbits                                                  (abs)        000477
_PWM2GIR                                                      (abs)        000476
_PWM2GIRbits                                                  (abs)        000476
_PWM2LDS                                                      (abs)        000471
_PWM2PIPOS                                                    (abs)        000475
_PWM2PRH                                                      (abs)        000473
_PWM2PRL                                                      (abs)        000472
_PWM2S1CFG                                                    (abs)        000479
_PWM2S1P1H                                                    (abs)        00047B
_PWM2S1P1L                                                    (abs)        00047A
_PWM2S1P2H                                                    (abs)        00047D
_PWM2S1P2L                                                    (abs)        00047C
_PWM2_16BIT_Enable                                            text20       0007E4
_PWM2_16BIT_Initialize                                        text6        00026A
_PWM2_16BIT_Period_DefaultInterruptHandler                    (abs)        000000
_PWM2_16BIT_Period_InterruptHandler                           nvCOMRAM     00051B
_PWM2_16BIT_Period_SetInterruptHandler                        text9        00073A
_PWM2_16BIT_Slice1Output1_DefaultInterruptHandler             (abs)        000000
_PWM2_16BIT_Slice1Output1_InterruptHandler                    nvCOMRAM     00051F
_PWM2_16BIT_Slice1Output1_SetInterruptHandler                 text8        000730
_PWM2_16BIT_Slice1Output2_DefaultInterruptHandler             (abs)        000000
_PWM2_16BIT_Slice1Output2_InterruptHandler                    nvCOMRAM     00051D
_PWM2_16BIT_Slice1Output2_SetInterruptHandler                 text7        000726
_PWM3CLK                                                      (abs)        00047F
_PWM3CON                                                      (abs)        000487
_PWM3CONbits                                                  (abs)        000487
_PWM3CPRE                                                     (abs)        000483
_PWM3ERS                                                      (abs)        00047E
_PWM3GIE                                                      (abs)        000486
_PWM3GIEbits                                                  (abs)        000486
_PWM3GIR                                                      (abs)        000485
_PWM3GIRbits                                                  (abs)        000485
_PWM3LDS                                                      (abs)        000480
_PWM3PIPOS                                                    (abs)        000484
_PWM3PRH                                                      (abs)        000482
_PWM3PRL                                                      (abs)        000481
_PWM3S1CFG                                                    (abs)        000488
_PWM3S1P1H                                                    (abs)        00048A
_PWM3S1P1L                                                    (abs)        000489
_PWM3S1P2H                                                    (abs)        00048C
_PWM3S1P2L                                                    (abs)        00048B
_PWM3_16BIT_Enable                                            text19       0007E0
_PWM3_16BIT_Initialize                                        text2        0001FC
_PWM3_16BIT_Period_DefaultInterruptHandler                    (abs)        000000
_PWM3_16BIT_Period_InterruptHandler                           nvCOMRAM     000521
_PWM3_16BIT_Period_SetInterruptHandler                        text5        00071C
_PWM3_16BIT_Slice1Output1_DefaultInterruptHandler             (abs)        000000
_PWM3_16BIT_Slice1Output1_InterruptHandler                    nvCOMRAM     000525
_PWM3_16BIT_Slice1Output1_SetInterruptHandler                 text4        000712
_PWM3_16BIT_Slice1Output2_DefaultInterruptHandler             (abs)        000000
_PWM3_16BIT_Slice1Output2_InterruptHandler                    nvCOMRAM     000523
_PWM3_16BIT_Slice1Output2_SetInterruptHandler                 text3        000708
_PWMIN0PPS                                                    (abs)        000257
_PWMIN1PPS                                                    (abs)        000258
_RA0PPS                                                       (abs)        000201
_RA1PPS                                                       (abs)        000202
_RC0PPS                                                       (abs)        000211
_RC1PPS                                                       (abs)        000212
_RC2PPS                                                       (abs)        000213
_RC3PPS                                                       (abs)        000214
_RC4PPS                                                       (abs)        000215
_RC5PPS                                                       (abs)        000216
_SLRCONA                                                      (abs)        000403
_SLRCONC                                                      (abs)        000413
_SYSTEM_Initialize                                            text1        0005CC
_TRISA                                                        (abs)        0004C6
_TRISC                                                        (abs)        0004C8
_WPUA                                                         (abs)        000401
_WPUC                                                         (abs)        000411
__HRAM                                                        (abs)        000000
__H__absolute__                                               __absolute__ 000000
__Habs1                                                       abs1         000000
__Hbank10                                                     bank10       000000
__Hbank11                                                     bank11       000000
__Hbank12                                                     bank12       000000
__Hbank13                                                     bank13       000000
__Hbank14                                                     bank14       000000
__Hbank15                                                     bank15       000000
__Hbank16                                                     bank16       000000
__Hbank17                                                     bank17       000000
__Hbank18                                                     bank18       000000
__Hbank19                                                     bank19       000000
__Hbank20                                                     bank20       000000
__Hbank5                                                      bank5        000000
__Hbank6                                                      bank6        000000
__Hbank7                                                      bank7        000000
__Hbank8                                                      bank8        000000
__Hbank9                                                      bank9        000000
__Hbigbss                                                     bigbss       000000
__Hbigdata                                                    bigdata      000000
__Hbigram                                                     bigram       000000
__Hbigsfr                                                     bigsfr       000000
__Hbss                                                        bss          000000
__HbssCOMRAM                                                  bssCOMRAM    000000
__Hcinit                                                      cinit        000000
__Hclrtext                                                    clrtext      000000
__Hcomram                                                     comram       000000
__Hconfig                                                     config       300009
__Hconst                                                      const        000000
__HcstackCOMRAM                                               cstackCOMRAM 000000
__Hdata                                                       data         000000
__Heeprom_data                                                eeprom_data  000000
__Hfarbss                                                     farbss       000000
__Hfardata                                                    fardata      000000
__Hheap                                                       heap         000000
__Hibigdata                                                   ibigdata     000000
__Hidata                                                      idata        000000
__Hidloc                                                      idloc        000000
__Hifardata                                                   ifardata     000000
__Hinit                                                       init         00001E
__Hintsave_regs                                               intsave_regs 000000
__Hirdata                                                     irdata       000000
__Hivt0x8                                                     ivt0x8       00001A
__Hmediumconst                                                mediumconst  000000
__HnvCOMRAM                                                   nvCOMRAM     000000
__HnvFARRAM                                                   nvFARRAM     000000
__Hnvbit                                                      nvbit        000000
__Hnvrram                                                     nvrram       000000
__Hparam                                                      rparam       000000
__Hpowerup                                                    powerup      000000
__Hram                                                        ram          000000
__Hramtop                                                     ramtop       001600
__Hrbit                                                       rbit         000000
__Hrbss                                                       rbss         000000
__Hrdata                                                      rdata        000000
__Hreset_vec                                                  reset_vec    000004
__Hrparam                                                     rparam       000000
__Hsfr                                                        sfr          000000
__Hsmallconst                                                 smallconst   000000
__Hspace_0                                                    (abs)        001600
__Hspace_1                                                    (abs)        000531
__Hspace_2                                                    (abs)        000000
__Hspace_4                                                    (abs)        600009
__Hstack                                                      stack        000000
__Hstruct                                                     struct       000000
__Htemp                                                       temp         000000
__Htext                                                       text         000000
__Htext0                                                      text0        000000
__Htext1                                                      text1        000000
__Htext10                                                     text10       000000
__Htext11                                                     text11       000000
__Htext12                                                     text12       000000
__Htext13                                                     text13       000000
__Htext14                                                     text14       000000
__Htext15                                                     text15       000000
__Htext16                                                     text16       000000
__Htext17                                                     text17       000000
__Htext18                                                     text18       000000
__Htext19                                                     text19       000000
__Htext2                                                      text2        000000
__Htext20                                                     text20       000000
__Htext21                                                     text21       000000
__Htext22                                                     text22       000000
__Htext23                                                     text23       000000
__Htext24                                                     text24       000000
__Htext25                                                     text25       000000
__Htext26                                                     text26       000000
__Htext27                                                     text27       000000
__Htext28                                                     text28       000000
__Htext29                                                     text29       000000
__Htext3                                                      text3        000000
__Htext30                                                     text30       000000
__Htext31                                                     text31       000000
__Htext32                                                     text32       000000
__Htext33                                                     text33       000000
__Htext34                                                     text34       000000
__Htext35                                                     text35       000000
__Htext36                                                     text36       000000
__Htext37                                                     text37       000000
__Htext38                                                     text38       000000
__Htext39                                                     text39       000000
__Htext4                                                      text4        000000
__Htext40                                                     text40       000000
__Htext41                                                     text41       000000
__Htext42                                                     text42       000000
__Htext43                                                     text43       000000
__Htext44                                                     text44       000000
__Htext45                                                     text45       000000
__Htext46                                                     text46       000000
__Htext47                                                     text47       000000
__Htext48                                                     text48       000000
__Htext49                                                     text49       000000
__Htext5                                                      text5        000000
__Htext50                                                     text50       000000
__Htext51                                                     text51       000000
__Htext52                                                     text52       000000
__Htext53                                                     text53       000000
__Htext54                                                     text54       000000
__Htext55                                                     text55       000000
__Htext6                                                      text6        000000
__Htext7                                                      text7        000000
__Htext8                                                      text8        000000
__Htext9                                                      text9        000000
__LRAM                                                        (abs)        000001
__L__absolute__                                               __absolute__ 000000
__Labs1                                                       abs1         000000
__Lbank10                                                     bank10       000000
__Lbank11                                                     bank11       000000
__Lbank12                                                     bank12       000000
__Lbank13                                                     bank13       000000
__Lbank14                                                     bank14       000000
__Lbank15                                                     bank15       000000
__Lbank16                                                     bank16       000000
__Lbank17                                                     bank17       000000
__Lbank18                                                     bank18       000000
__Lbank19                                                     bank19       000000
__Lbank20                                                     bank20       000000
__Lbank5                                                      bank5        000000
__Lbank6                                                      bank6        000000
__Lbank7                                                      bank7        000000
__Lbank8                                                      bank8        000000
__Lbank9                                                      bank9        000000
__Lbigbss                                                     bigbss       000000
__Lbigdata                                                    bigdata      000000
__Lbigram                                                     bigram       000000
__Lbigsfr                                                     bigsfr       000000
__Lbss                                                        bss          000000
__LbssCOMRAM                                                  bssCOMRAM    000000
__Lcinit                                                      cinit        000000
__Lclrtext                                                    clrtext      000000
__Lcomram                                                     comram       000000
__Lconfig                                                     config       000000
__Lconst                                                      const        000000
__LcstackCOMRAM                                               cstackCOMRAM 000000
__Ldata                                                       data         000000
__Leeprom_data                                                eeprom_data  000000
__Lfarbss                                                     farbss       000000
__Lfardata                                                    fardata      000000
__Lheap                                                       heap         000000
__Libigdata                                                   ibigdata     000000
__Lidata                                                      idata        000000
__Lidloc                                                      idloc        000000
__Lifardata                                                   ifardata     000000
__Linit                                                       init         00001A
__Lintsave_regs                                               intsave_regs 000000
__Lirdata                                                     irdata       000000
__Livt0x8                                                     ivt0x8       000008
__Lmediumconst                                                mediumconst  000000
__LnvCOMRAM                                                   nvCOMRAM     000000
__LnvFARRAM                                                   nvFARRAM     000000
__Lnvbit                                                      nvbit        000000
__Lnvrram                                                     nvrram       000000
__Lparam                                                      rparam       000000
__Lpowerup                                                    powerup      000000
__Lram                                                        ram          000000
__Lramtop                                                     ramtop       001600
__Lrbit                                                       rbit         000000
__Lrbss                                                       rbss         000000
__Lrdata                                                      rdata        000000
__Lreset_vec                                                  reset_vec    000000
__Lrparam                                                     rparam       000000
__Lsfr                                                        sfr          000000
__Lsmallconst                                                 smallconst   000000
__Lspace_0                                                    (abs)        000000
__Lspace_1                                                    (abs)        000000
__Lspace_2                                                    (abs)        000000
__Lspace_4                                                    (abs)        000000
__Lstack                                                      stack        000000
__Lstruct                                                     struct       000000
__Ltemp                                                       temp         000000
__Ltext                                                       text         000000
__Ltext0                                                      text0        000000
__Ltext1                                                      text1        000000
__Ltext10                                                     text10       000000
__Ltext11                                                     text11       000000
__Ltext12                                                     text12       000000
__Ltext13                                                     text13       000000
__Ltext14                                                     text14       000000
__Ltext15                                                     text15       000000
__Ltext16                                                     text16       000000
__Ltext17                                                     text17       000000
__Ltext18                                                     text18       000000
__Ltext19                                                     text19       000000
__Ltext2                                                      text2        000000
__Ltext20                                                     text20       000000
__Ltext21                                                     text21       000000
__Ltext22                                                     text22       000000
__Ltext23                                                     text23       000000
__Ltext24                                                     text24       000000
__Ltext25                                                     text25       000000
__Ltext26                                                     text26       000000
__Ltext27                                                     text27       000000
__Ltext28                                                     text28       000000
__Ltext29                                                     text29       000000
__Ltext3                                                      text3        000000
__Ltext30                                                     text30       000000
__Ltext31                                                     text31       000000
__Ltext32                                                     text32       000000
__Ltext33                                                     text33       000000
__Ltext34                                                     text34       000000
__Ltext35                                                     text35       000000
__Ltext36                                                     text36       000000
__Ltext37                                                     text37       000000
__Ltext38                                                     text38       000000
__Ltext39                                                     text39       000000
__Ltext4                                                      text4        000000
__Ltext40                                                     text40       000000
__Ltext41                                                     text41       000000
__Ltext42                                                     text42       000000
__Ltext43                                                     text43       000000
__Ltext44                                                     text44       000000
__Ltext45                                                     text45       000000
__Ltext46                                                     text46       000000
__Ltext47                                                     text47       000000
__Ltext48                                                     text48       000000
__Ltext49                                                     text49       000000
__Ltext5                                                      text5        000000
__Ltext50                                                     text50       000000
__Ltext51                                                     text51       000000
__Ltext52                                                     text52       000000
__Ltext53                                                     text53       000000
__Ltext54                                                     text54       000000
__Ltext55                                                     text55       000000
__Ltext6                                                      text6        000000
__Ltext7                                                      text7        000000
__Ltext8                                                      text8        000000
__Ltext9                                                      text9        000000
__S0                                                          (abs)        0007EC
__S1                                                          (abs)        000531
__S4                                                          (abs)        000000
__S5                                                          (abs)        000000
___heap_hi                                                    (abs)        000000
___heap_lo                                                    (abs)        000000
___inthi_sp                                                   stack        000000
___intlo_sp                                                   stack        000000
___param_bank                                                 (abs)        000000
___rparam_used                                                (abs)        000001
___sp                                                         stack        000000
__accesstop                                                   (abs)        000560
__activetblptr                                                (abs)        000002
__end_of_I2C1_Initialize                                      text18       000642
__end_of_I2C1_Isr                                             text36       000150
__end_of_I2C1_Open                                            text24       000476
__end_of_I2C1_SlaveAddrCallBack                               text52       0005A8
__end_of_I2C1_SlaveClearBuff                                  text51       0007DC
__end_of_I2C1_SlaveClearIrq                                   text50       0007AE
__end_of_I2C1_SlaveDefAddrInterruptHandler                    text53       0007B6
__end_of_I2C1_SlaveDefRdInterruptHandler                      text43       00051E
__end_of_I2C1_SlaveDefWrInterruptHandler                      text38       000418
__end_of_I2C1_SlaveEnableIrq                                  text34       0006FA
__end_of_I2C1_SlaveGetAddr                                    text54       0007BE
__end_of_I2C1_SlaveGetRxData                                  text44       0007D6
__end_of_I2C1_SlaveIsAddr                                     text49       0006B0
__end_of_I2C1_SlaveIsRead                                     text48       00069A
__end_of_I2C1_SlaveIsRxBufFull                                text47       000684
__end_of_I2C1_SlaveIsStop                                     text46       00066E
__end_of_I2C1_SlaveIsTxBufEmpty                               text45       000658
__end_of_I2C1_SlaveOpen                                       text33       0006C4
__end_of_I2C1_SlaveRdCallBack                                 text42       00057A
__end_of_I2C1_SlaveReleaseClock                               text41       0007D0
__end_of_I2C1_SlaveSendTxData                                 text39       0007A6
__end_of_I2C1_SlaveSetAddrIntHandler                          text32       00079E
__end_of_I2C1_SlaveSetBusColIntHandler                        text31       000794
__end_of_I2C1_SlaveSetCounter                                 text40       000708
__end_of_I2C1_SlaveSetIsrHandler                              text30       00078A
__end_of_I2C1_SlaveSetReadIntHandler                          text29       000780
__end_of_I2C1_SlaveSetSlaveAddr                               text28       0006E8
__end_of_I2C1_SlaveSetSlaveMask                               text27       0006D6
__end_of_I2C1_SlaveSetWrColIntHandler                         text26       000776
__end_of_I2C1_SlaveSetWriteIntHandler                         text25       00076C
__end_of_I2C1_SlaveWrCallBack                                 text37       00054C
__end_of_I2C1_ZeroBuff                                        text23       0007CA
__end_of_I2C1_ZeroBuffer                                      text22       0007C4
__end_of_INTERRUPT_Initialize                                 text17       0007E0
__end_of_INTERRUPT_InterruptManager                           text35       0001FC
__end_of_OSCILLATOR_Initialize                                text16       000626
__end_of_PIN_MANAGER_Initialize                               text15       0003B4
__end_of_PMD_Initialize                                       text14       00060A
__end_of_PWM1_16BIT_Enable                                    text21       0007EC
__end_of_PWM1_16BIT_Initialize                                text10       000346
__end_of_PWM1_16BIT_Period_SetInterruptHandler                text13       000762
__end_of_PWM1_16BIT_Slice1Output1_SetInterruptHandler         text12       000758
__end_of_PWM1_16BIT_Slice1Output2_SetInterruptHandler         text11       00074E
__end_of_PWM2_16BIT_Enable                                    text20       0007E8
__end_of_PWM2_16BIT_Initialize                                text6        0002D8
__end_of_PWM2_16BIT_Period_SetInterruptHandler                text9        000744
__end_of_PWM2_16BIT_Slice1Output1_SetInterruptHandler         text8        00073A
__end_of_PWM2_16BIT_Slice1Output2_SetInterruptHandler         text7        000730
__end_of_PWM3_16BIT_Enable                                    text19       0007E4
__end_of_PWM3_16BIT_Initialize                                text2        00026A
__end_of_PWM3_16BIT_Period_SetInterruptHandler                text5        000726
__end_of_PWM3_16BIT_Slice1Output1_SetInterruptHandler         text4        00071C
__end_of_PWM3_16BIT_Slice1Output2_SetInterruptHandler         text3        000712
__end_of_SYSTEM_Initialize                                    text1        0005EE
__end_of__initialization                                      cinit        0005C2
__end_of_main                                                 text0        0004CE
__initialization                                              cinit        0005A8
__mediumconst                                                 mediumconst  000000
__pbssCOMRAM                                                  bssCOMRAM    000501
__pcinit                                                      cinit        0005A8
__pcstackCOMRAM                                               cstackCOMRAM 000527
__pivt0x8                                                     ivt0x8       000008
__pnvCOMRAM                                                   nvCOMRAM     000515
__ptext0                                                      text0        000476
__ptext1                                                      text1        0005CC
__ptext10                                                     text10       0002D8
__ptext11                                                     text11       000744
__ptext12                                                     text12       00074E
__ptext13                                                     text13       000758
__ptext14                                                     text14       0005EE
__ptext15                                                     text15       000346
__ptext16                                                     text16       00060A
__ptext17                                                     text17       0007DC
__ptext18                                                     text18       000626
__ptext19                                                     text19       0007E0
__ptext2                                                      text2        0001FC
__ptext20                                                     text20       0007E4
__ptext21                                                     text21       0007E8
__ptext22                                                     text22       0007BE
__ptext23                                                     text23       0007C4
__ptext24                                                     text24       000418
__ptext25                                                     text25       000762
__ptext26                                                     text26       00076C
__ptext27                                                     text27       0006C4
__ptext28                                                     text28       0006D6
__ptext29                                                     text29       000776
__ptext3                                                      text3        000708
__ptext30                                                     text30       000780
__ptext31                                                     text31       00078A
__ptext32                                                     text32       000794
__ptext33                                                     text33       0006B0
__ptext34                                                     text34       0006E8
__ptext35                                                     text35       000150
__ptext36                                                     text36       00001E
__ptext37                                                     text37       00051E
__ptext38                                                     text38       0003B4
__ptext39                                                     text39       00079E
__ptext4                                                      text4        000712
__ptext40                                                     text40       0006FA
__ptext41                                                     text41       0007CA
__ptext42                                                     text42       00054C
__ptext43                                                     text43       0004CE
__ptext44                                                     text44       0007D0
__ptext45                                                     text45       000642
__ptext46                                                     text46       000658
__ptext47                                                     text47       00066E
__ptext48                                                     text48       000684
__ptext49                                                     text49       00069A
__ptext5                                                      text5        00071C
__ptext50                                                     text50       0007A6
__ptext51                                                     text51       0007D6
__ptext52                                                     text52       00057A
__ptext53                                                     text53       0007AE
__ptext54                                                     text54       0007B6
__ptext55                                                     text55       000000
__ptext6                                                      text6        00026A
__ptext7                                                      text7        000726
__ptext8                                                      text8        000730
__ptext9                                                      text9        00073A
__ramtop                                                      ramtop       001600
__smallconst                                                  smallconst   000000
_i2c1RdBuf                                                    bssCOMRAM    000501
_i2c1RdData                                                   bssCOMRAM    000513
_i2c1SlaveAddr                                                bssCOMRAM    000512
_i2c1SlaveState                                               bssCOMRAM    000511
_i2c1WrData                                                   bssCOMRAM    000514
_main                                                         text0        000476
end_of_initialization                                         cinit        0005C2
intlevel0                                                     text         000000
intlevel1                                                     text         000000
intlevel2                                                     text         000000
intlevel3                                                     text         000000
isa$std                                                       (abs)        000001
isa$xinst                                                     (abs)        000000
ivt0x8_base                                                   ivt0x8       000008
main@SlaveIsStop                                              cstackCOMRAM 000530
stackhi                                                       (abs)        000000
stacklo                                                       (abs)        000000
start                                                         init         00001A
start_initialization                                          cinit        0005A8


MODULE INFORMATION

Module		Function		Class		Link	Load	Size
mcc_generated_files/pwm2_16bit.c
		_PWM2_16BIT_Period_SetInterruptHandler		CODE           	073A	0000	10
		_PWM2_16BIT_Slice1Output1_SetInterruptHandler		CODE           	0730	0000	10
		_PWM2_16BIT_Slice1Output2_SetInterruptHandler		CODE           	0726	0000	10
		_PWM2_16BIT_Initialize		CODE           	026A	0000	110
		_PWM2_16BIT_Enable		CODE           	07E4	0000	4

mcc_generated_files/pwm2_16bit.c estimated size: 144

mcc_generated_files/interrupt_manager.c
		_INTERRUPT_Initialize		CODE           	07DC	0000	4
		_INTERRUPT_InterruptManager		CODE           	0150	0000	172

mcc_generated_files/interrupt_manager.c estimated size: 176

mcc_generated_files/pin_manager.c
		_PIN_MANAGER_Initialize		CODE           	0346	0000	110

mcc_generated_files/pin_manager.c estimated size: 110

mcc_generated_files/i2c1_slave.c
		_I2C1_SlaveSetReadIntHandler		CODE           	0776	0000	10
		_I2C1_SlaveDefAddrInterruptHandler		CODE           	07AE	0000	8
		_I2C1_SlaveSetCounter		CODE           	06FA	0000	14
		_I2C1_SlaveSetAddrIntHandler		CODE           	0794	0000	10
		_I2C1_SlaveIsRead		CODE           	0684	0000	22
		_I2C1_SlaveSetIsrHandler		CODE           	0780	0000	10
		_I2C1_SlaveIsAddr		CODE           	069A	0000	22
		_I2C1_ZeroBuffer		CODE           	07BE	0000	6
		_I2C1_SlaveIsStop		CODE           	0658	0000	22
		_I2C1_SlaveEnableIrq		CODE           	06E8	0000	18
		_I2C1_SlaveDefRdInterruptHandler		CODE           	04CE	0000	80
		_I2C1_SlaveDefWrInterruptHandler		CODE           	03B4	0000	100
		_I2C1_SlaveGetAddr		CODE           	07B6	0000	8
		_I2C1_SlaveOpen		CODE           	06B0	0000	20
		_I2C1_SlaveSendTxData		CODE           	079E	0000	8
		_I2C1_SlaveSetSlaveAddr		CODE           	06D6	0000	18
		_I2C1_SlaveRdCallBack		CODE           	054C	0000	46
		_I2C1_SlaveWrCallBack		CODE           	051E	0000	46
		_I2C1_Isr      		CODE           	001E	0000	306
		_I2C1_Open     		CODE           	0418	0000	94
		_I2C1_SlaveAddrCallBack		CODE           	057A	0000	46
		_I2C1_Initialize		CODE           	0626	0000	28
		_I2C1_SlaveSetWrColIntHandler		CODE           	076C	0000	10
		_I2C1_SlaveIsTxBufEmpty		CODE           	0642	0000	22
		_I2C1_SlaveIsRxBufFull		CODE           	066E	0000	22
		_I2C1_SlaveClearIrq		CODE           	07A6	0000	8
		_I2C1_SlaveGetRxData		CODE           	07D0	0000	6
		_I2C1_SlaveSetWriteIntHandler		CODE           	0762	0000	10
		_I2C1_SlaveSetBusColIntHandler		CODE           	078A	0000	10
		_I2C1_SlaveReleaseClock		CODE           	07CA	0000	6
		_I2C1_ZeroBuff 		CODE           	07C4	0000	6
		_I2C1_SlaveSetSlaveMask		CODE           	06C4	0000	18
		_I2C1_SlaveClearBuff		CODE           	07D6	0000	6

mcc_generated_files/i2c1_slave.c estimated size: 1066

mcc_generated_files/pwm1_16bit.c
		_PWM1_16BIT_Period_SetInterruptHandler		CODE           	0758	0000	10
		_PWM1_16BIT_Slice1Output1_SetInterruptHandler		CODE           	074E	0000	10
		_PWM1_16BIT_Slice1Output2_SetInterruptHandler		CODE           	0744	0000	10
		_PWM1_16BIT_Initialize		CODE           	02D8	0000	110
		_PWM1_16BIT_Enable		CODE           	07E8	0000	4

mcc_generated_files/pwm1_16bit.c estimated size: 144

shared
		__initialization		CODE           	05A8	0000	26

shared estimated size: 26

mcc_generated_files/mcc.c
		_PMD_Initialize		CODE           	05EE	0000	28
		_OSCILLATOR_Initialize		CODE           	060A	0000	28
		_SYSTEM_Initialize		CODE           	05CC	0000	34

mcc_generated_files/mcc.c estimated size: 90

mcc_generated_files/pwm3_16bit.c
		_PWM3_16BIT_Enable		CODE           	07E0	0000	4
		_PWM3_16BIT_Period_SetInterruptHandler		CODE           	071C	0000	10
		_PWM3_16BIT_Slice1Output1_SetInterruptHandler		CODE           	0712	0000	10
		_PWM3_16BIT_Slice1Output2_SetInterruptHandler		CODE           	0708	0000	10
		_PWM3_16BIT_Initialize		CODE           	01FC	0000	110

mcc_generated_files/pwm3_16bit.c estimated size: 144

main.c
		_main          		CODE           	0476	0000	88

main.c estimated size: 88

